:10000000000000000000B228AA004230A1000F301A
:10001000A200692003191210031D1214FC3E031CD8
:100020009210031892144030A1004230A2000F3009
:10003000A500A60112183A2092183A206B2021033D
:100040008316920083122108A3002208A40020082E
:10005000A700A800200FA8019820260895000C30C2
:100060009700A51B9716251B1716831606118312DA
:100070001215AE283B200310A50CA20CA10C080001
:1000800083178001840AFF3E031D4128AE28A40186
:10009000A300FF30A307031CA407031CAE28000025
:1000A000A201003055204928A201E83EA100A20982
:1000B000FC30031C5E28A10703185B28A107000081
:1000C000A20F5B2821186428A11C6828000068285A
:1000D0000800A601A5011030A700220DA50DA60D50
:1000E0002308A5022408031C240FA60203187F2856
:1000F0002308A50724080318240FA6070310A10D41
:10010000A20DA70B6D2821080800A300A400A201DE
:100110000830A700A10DA20D23082202031C93287A
:100120002308A2020314A40DA70B8A2824080800A0
:100130001030AD00A201A101A80CA70C031CA62839
:100140002308A10724080318240FA207A20CA10C5E
:10015000A60CA50CAD0B9C28250808008313831260
:1001600003130800830107309F00A001A400D030D2
:10017000A30001300420803085003A3083168500CA
:10018000F7308600811320308400603083124120D4
:10019000A030840050304120203084003030402096
:1001A000F628013030180030AE00FF302F02013049
:1001B00003180030AE040319F528301CE128AF0AFB
:1001C000E228AF032F08A0000730A400D030A3001E
:1001D000013004202F08A1000A30852001390319BD
:1001E0000511031D0515143047200800050C0318E0
:1001F0000515031C05110618FE28FB2805304720AD
:10020000061C032900290530472005140130B006DB
:10021000FA304720061C2A29003030180130AE0081
:100220000B302F02031816290301031D0130AE0401
:1002300003192829D120013006180030AE002F0AFA
:100240000130031D0030AE0403192729F6280C29BC
:1002500005103D2906183D29D12001303018003005
:10026000AE000B302F02031C37290301031D0130A0
:0E027000AE0503193C293D292A29F6283E290E
:02400E00503F21
:00000001FF
